:020000040800F2
:1000000000C00020B5450008894500088D4500085E
:10001000914500089545000899450008000000003A
:100020000000000000000000000000009D450008E6
:10003000A145000800000000A5450008A9450008EA
:10004000FD450008FD450008FD450008FD45000888
:10005000FD450008FD450008FD450008FD45000878
:10006000FD450008FD450008FD450008F93D000874
:10007000FD450008FD450008FD450008FD45000858
:10008000FD450008FD450008FD450008FD45000848
:10009000FD450008FD450008FD450008FD45000838
:1000A000FD450008FD450008FD450008FD45000828
:1000B000FD450008FD450008FD450008FD45000818
:1000C000FD450008FD450008FD450008FD45000808
:1000D000FD450008FD450008FD450008FD450008F8
:1000E000FD450008FD450008FD450008FD450008E8
:1000F000FD450008FD450008FD450008FD450008D8
:10010000FD450008FD450008FD450008FD450008C7
:10011000FD450008FD450008FD450008FD450008B7
:10012000FD450008FD450008FD450008FD450008A7
:1001300000000000000000000000000000000000BF
:1001400000000000000000000000000000000000AF
:10015000000000000000000000000000000000009F
:10016000000000000000000000000000000000008F
:10017000000000000000000000000000000000007F
:10018000000000000000000000000000000000006F
:10019000000000000000000000000000000000005F
:1001A000000000000000000000000000000000004F
:1001B000000000000000000000000000000000003F
:1001C000000000000000000000000000000000002F
:1001D000000000000000000000000000000000001F
:0401E0005FF8E0F1F3
:1001E800044B05481B1A062B02D9044B03B11847C8
:1001F800704700BF8B00002088000020000000002E
:1002080005490648091A891001EBD171491002D035
:10021800034B03B11847704788000020880000206E
:100228000000000010B5064C237843B9FFF7D8FF4B
:10023800044B13B10448AFF300800123237010BDB1
:100248008800002000000000B04E000808B5084BE8
:100258001BB108480849AFF300800848036813B980
:10026800BDE80840CCE7064B002BF9D09847F7E7E4
:1002780000000000B04E00088C000020880000201C
:100288000000000081F0004102E000BF83F000435D
:1002980030B54FEA41044FEA430594EA050F08BF19
:1002A80090EA020F1FBF54EA000C55EA020C7FEADD
:1002B800645C7FEA655C00F0E2804FEA5454D4EB5A
:1002C8005555B8BF6D420CDD2C4480EA020281EA24
:1002D800030382EA000083EA010180EA020281EA5C
:1002E8000303362D88BF30BD11F0004F4FEA0131AE
:1002F8004FF4801C4CEA113102D0404261EB4101BD
:1003080013F0004F4FEA03334CEA133302D0524242
:1003180063EB430394EA050F00F0A780A4F10104FE
:10032800D5F1200E0DDB02FA0EFC22FA05F2801838
:1003380041F1000103FA0EF2801843FA05F359411E
:100348000EE0A5F120050EF1200E012A03FA0EFC9D
:1003580028BF4CF0020C43FA05F3C01851EBE371C7
:1003680001F0004507D54FF0000EDCF1000C7EEBE4
:1003780000006EEB0101B1F5801F1BD3B1F5001F22
:100388000CD349085FEA30004FEA3C0C04F1010441
:100398004FEA445212F5800F80F09A80BCF1004F6A
:1003A80008BF5FEA500C50F1000041EB045141EAEC
:1003B800050130BD5FEA4C0C404141EB010111F4ED
:1003C800801FA4F10104E9D191F0000F04BF014698
:1003D8000020B1FA81F308BF2033A3F10B03B3F176
:1003E80020020CDA0C3208DD02F1140CC2F10C0206
:1003F80001FA0CF021FA02F10CE002F11402D8BF64
:10040800C2F1200C01FA02F120FA0CFCDCBF41EA2F
:100418000C019040E41AA2BF01EB0451294330BDFE
:100428006FEA04041F3C1CDA0C340EDC04F11404DB
:10043800C4F1200220FA04F001FA02F340EA0300B2
:1004480021FA04F345EA030130BDC4F10C04C4F1F8
:10045800200220FA02F001FA04F340EA03002946D8
:1004680030BD21FA04F0294630BD94F0000F83F422
:10047800801306BF81F480110134013D4EE77FEA05
:10048800645C18BF7FEA655C29D094EA050F08BF51
:1004980090EA020F05D054EA000C04BF1946104632
:1004A80030BD91EA030F1EBF0021002030BD5FEA76
:1004B800545C05D14000494128BF41F0004130BD9E
:1004C80014F580043CBF01F5801130BD01F00045F2
:1004D80045F0FE4141F470014FF0000030BD7FEA65
:1004E800645C1ABF194610467FEA655C1CBF0B4660
:1004F800024650EA013406BF52EA033591EA030F77
:1005080041F4002130BD00BF90F0000F04BF00216E
:10051800704730B54FF4806404F132044FF00005A1
:100528004FF0000150E700BF90F0000F04BF00211A
:10053800704730B54FF4806404F1320410F0004580
:1005480048BF40424FF000013EE700BF42004FEA7B
:10055800E2014FEA31014FEA02701FBF12F07F43F8
:1005680093F07F4F81F06051704792F0000F14BFF5
:1005780093F07F4F704730B54FF4607401F0004539
:1005880021F0004120E700BF50EA010208BF704790
:1005980030B54FF000050AE050EA010208BF704785
:1005A80030B511F0004502D5404261EB41014FF4EE
:1005B800806404F132045FEA915C3FF4DCAE4FF0F2
:1005C80003025FEADC0C18BF03325FEADC0C18BFD9
:1005D800033202EBDC02C2F1200300FA03FC20FA2A
:1005E80002F001FA03FE40EA0E0021FA02F1144477
:1005F800C1E600BF70B54FF0FF0C4CF4E06C1CEA8C
:1006080011541DBF1CEA135594EA0C0F95EA0C0F00
:1006180000F0DEF82C4481EA030621EA4C5123EA73
:100628004C5350EA013518BF52EA033541F48011A2
:1006380043F4801338D0A0FB02CE4FF00005E1FB55
:1006480002E506F00042E0FB03E54FF00006E1FB9F
:1006580003569CF0000F18BF4EF0010EA4F1FF04E2
:10066800B6F5007F64F5407404D25FEA4E0E6D4122
:1006780046EB060642EAC62141EA55514FEAC52033
:1006880040EA5E504FEACE2EB4F1FD0C88BFBCF5AF
:10069800E06F1ED8BEF1004F08BF5FEA500E50F160
:1006A800000041EB045170BD06F0004646EA010126
:1006B80040EA020081EA0301B4EB5C04C2BFD4EB58
:1006C8000C0541EA045170BD41F480114FF0000E51
:1006D800013C00F3AB8014F1360FDEBF002001F0BF
:1006E800004170BDC4F10004203C35DA0C341BDC39
:1006F80004F11404C4F1200500FA05F320FA04F00B
:1007080001FA05F240EA020001F0004221F000413E
:1007180010EBD37021FA04F642EB06015EEA430EB1
:1007280008BF20EAD37070BDC4F10C04C4F12005E1
:1007380000FA04F320FA05F001FA04F240EA020094
:1007480001F0004110EBD37041F100015EEA430E65
:1007580008BF20EAD37070BDC4F1200500FA05F285
:100768004EEA020E20FA04F301FA05F243EA020304
:1007780021FA04F001F0004121FA04F220EA020013
:1007880000EBD3705EEA430E08BF20EAD37070BD59
:1007980094F0000F0FD101F00046400041EB010139
:1007A80011F4801F08BF013CF7D041EA060195F01B
:1007B800000F18BF704703F00046520043EB0303D5
:1007C80013F4801F08BF013DF7D043EA06037047C2
:1007D80094EA0C0F0CEA135518BF95EA0C0F0CD0CD
:1007E80050EA410618BF52EA4306D1D181EA030113
:1007F80001F000414FF0000070BD50EA410606BF0D
:100808001046194652EA430619D094EA0C0F02D151
:1008180050EA013613D195EA0C0F05D152EA033696
:100828001CBF104619460AD181EA030101F00041B4
:1008380041F0FE4141F470014FF0000070BD41F0FD
:10084800FE4141F4780170BD70B54FF0FF0C4CF4D7
:10085800E06C1CEA11541DBF1CEA135594EA0C0FF6
:1008680095EA0C0F00F0A7F8A4EB050481EA030E43
:1008780052EA03354FEA013100F088804FEA03332A
:100888004FF0805545EA131343EA12634FEA0222F8
:1008980045EA111545EA10654FEA00260EF00041B9
:1008A8009D4208BF964244F1FD0404F5407402D20B
:1008B8005B084FEA3202B61A65EB03055B084FEA9C
:1008C80032024FF480104FF4002CB6EB020E75EB99
:1008D800030E22BFB61A754640EA0C005B084FEAC1
:1008E8003202B6EB020E75EB030E22BFB61A75463E
:1008F80040EA5C005B084FEA3202B6EB020E75EB89
:10090800030E22BFB61A754640EA9C005B084FEA00
:100918003202B6EB020E75EB030E22BFB61A75460D
:1009280040EADC0055EA060E18D04FEA051545EAFC
:1009380016754FEA06164FEAC30343EA52734FEAA5
:10094800C2025FEA1C1CC0D111F4801F0BD141EA1E
:1009580000014FF000004FF0004CB6E711F4801F83
:1009680004BF01430020B4F1FD0C88BFBCF5E06F63
:100978003FF6AFAEB5EB030C04BFB6EB020C5FEA73
:10098800500C50F1000041EB045170BD0EF0004EC8
:100998004EEA113114EB5C04C2BFD4EB0C0541EAFA
:1009A800045170BD41F480114FF0000E013C90E6F7
:1009B80045EA060E8DE60CEA135594EA0C0F08BFBB
:1009C80095EA0C0F3FF43BAF94EA0C0F0AD150EABA
:1009D80001347FF434AF95EA0C0F7FF425AF10464D
:1009E80019462CE795EA0C0F06D152EA03353FF475
:1009F800FDAE1046194622E750EA410618BF52EAF2
:100A080043067FF4C5AE50EA41047FF40DAF52EAC5
:100A180043057FF4EBAE12E74FF0FF3C06E000BF62
:100A28004FF0010C02E000BF4FF0010C4DF804CD6F
:100A38004FEA410C7FEA6C5C4FEA430C18BF7FEA2F
:100A48006C5C1BD001B050EA410C0CBF52EA430C5D
:100A580091EA030F02BF90EA020F0020704710F1DD
:100A6800000F91EA030F58BF994208BF90422CBF6C
:100A7800D8176FEAE37040F0010070474FEA410C65
:100A88007FEA6C5C02D150EA013C07D14FEA430C83
:100A98007FEA6C5CD6D152EA033CD3D05DF8040BF4
:100AA800704700BF8446104662468C461946634626
:100AB80000E000BF01B5FFF7B7FF002848BF10F1FD
:100AC800000F01BD4DF808EDFFF7F4FF0CBF012042
:100AD80000205DF808FB00BF4DF808EDFFF7EAFFBE
:100AE80034BF012000205DF808FB00BF4DF808ED79
:100AF800FFF7E0FF94BF012000205DF808FB00BF6E
:100B08004DF808EDFFF7CEFF94BF012000205DF8F7
:100B180008FB00BF4DF808EDFFF7C4FF34BF012004
:100B280000205DF808FB00BF4FEA410212F50012F1
:100B380015D211D56FF47873B3EB625212D94FEA1C
:100B4800C12343F0004343EA505311F0004F23FA06
:100B580002F018BF404270474FF00000704750EA5B
:100B6800013005D111F0004008BF6FF00040704718
:100B78004FF00000704700BF4FEA4102B2F1E04376
:100B880024BFB3F5001CDCF1FE5C0DD901F0004C6C
:100B98004FEAC0024CEA5070B2F1004F40EB8300BC
:100BA80008BF20F00100704711F0804F21D113F1E8
:100BB8003872BCBF01F00040704741F480114FEA21
:100BC8005252C2F11802C2F1200C10FA0CF320FAAA
:100BD80002F018BF40F001004FEAC1234FEAD323C7
:100BE80003FA0CFC40EA0C0023FA02F34FEA430331
:100BF800CCE77FEA625307D150EA01331EBF4FF0BA
:100C0800FE4040F44000704701F0004040F0FE40D4
:100C180040F40000704700BF80F0004002E000BFD1
:100C280081F0004142001FBF5FEA410392EA030FCF
:100C38007FEA226C7FEA236C6AD04FEA1262D2EB19
:100C48001363C1BFD218414048404140B8BF5B421E
:100C5800192B88BF704710F0004F40F4000020F0B7
:100C68007F4018BF404211F0004F41F4000121F0CD
:100C78007F4118BF494292EA030F3FD0A2F1010217
:100C880041FA03FC10EB0C00C3F1200301FA03F155
:100C980000F0004302D5494260EB4000B0F5000F78
:100CA80013D3B0F1807F06D340084FEA310102F137
:100CB8000102FE2A51D2B1F1004F40EBC25008BFE9
:100CC80020F0010040EA03007047490040EB0000B3
:100CD80010F4000FA2F10102EDD1B0FA80FCACF1E2
:100CE800080CB2EB0C0200FA0CF0AABF00EBC250E1
:100CF80052421843BCBFD0401843704792F0000FCF
:100D080081F4000106BF80F400000132013BB5E721
:100D18004FEA41037FEA226C18BF7FEA236C21D097
:100D280092EA030F04D092F0000F08BF08467047FC
:100D380090EA010F1CBF0020704712F07F4F04D1CA
:100D4800400028BF40F00040704712F100723CBFDD
:100D580000F50000704700F0004343F0FE4040F407
:100D6800000070477FEA226216BF08467FEA2363C5
:100D78000146420206BF5FEA412390EA010F40F4B0
:100D8800800070474FF0000304E000BF10F00043FC
:100D980048BF40425FEA000C08BF704743F09643E3
:100DA80001464FF000001CE050EA010208BF7047FE
:100DB8004FF000030AE000BF50EA010208BF704785
:100DC80011F0004302D5404261EB41015FEA010C9A
:100DD80002BF84460146002043F0B64308BFA3F192
:100DE8008053A3F50003BCFA8CF2083AA3EBC25374
:100DF80010DB01FA02FC634400FA02FCC2F1200293
:100E0800BCF1004F20FA02F243EB020008BF20F0C9
:100E18000100704702F1200201FA02FCC2F120022F
:100E280050EA4C0021FA02F243EB020008BF20EA24
:100E3800DC7070474FF0FF3C06E000BF4FF0010C3C
:100E480002E000BF4FF0010C4DF804CD4FEA40021C
:100E58004FEA41037FEA226C18BF7FEA236C11D066
:100E680001B052EA530C18BF90EA010F58BFB2EB19
:100E7800030088BFC81738BF6FEAE17018BF40F099
:100E8800010070477FEA226C02D15FEA402C05D14D
:100E98007FEA236CE4D15FEA412CE1D05DF8040BD2
:100EA800704700BF844608466146FFE70FB5FFF765
:100EB800C9FF002848BF10F1000F0FBD4DF808ED1D
:100EC800FFF7F4FF0CBF012000205DF808FB00BF0E
:100ED8004DF808EDFFF7EAFF34BF012000205DF868
:100EE80008FB00BF4DF808EDFFF7E0FF94BF0120B5
:100EF80000205DF808FB00BF4DF808EDFFF7D2FFB2
:100F080094BF012000205DF808FB00BF4DF808EDF4
:100F1800FFF7C8FF34BF012000205DF808FB00BFC1
:100F280082B0084B1B68084AA2FB03235B0A00FB3C
:100F380003F0019000BF019B5A1E0192002BF9D1CA
:100F480002B0704700000020D34D621070B582B027
:100F58000446036813F0010F6BD0A84B5B6803F0DD
:100F68000C03042B0AD0A54B5B6803F00C03082B79
:100F78000DD1A24B5B6813F4803F08D09F4B1B68D0
:100F880013F4003F55D06368002B52D1B8E1636871
:100F9800B3F5803F05D1994A136843F48033136051
:100FA80026E063B903F1804303F504331A6822F499
:100FB80080321A601A6822F480221A6018E0B3F5A9
:100FC800A02F0CD103F18043A3F53C331A6842F4F7
:100FD80080221A601A6842F480321A6008E0874B4F
:100FE8001A6822F480321A601A6822F480221A6081
:100FF80063687BB101F01CF8054605E001F018F8BC
:10100800401B642800F27E817C4B1B6813F4003F70
:10101800F4D00EE001F00CF8054605E001F008F800
:10102800401B642800F27081744B1B6813F4003F66
:10103800F4D1236813F0020F50D0704B5B6813F0A3
:101048000C0F0AD06D4B5B6803F00C03082B16D10C
:101058006A4B5B6813F4803F11D1684B1B6813F02F
:10106800020F03D02369012B40F05081634A1368B3
:1010780023F0F803616943EAC10313602EE0236992
:10108800D3B101225E4B1A6000F0D2FF054605E09D
:1010980000F0CEFF401B022800F23A81574B1B6834
:1010A80013F0020FF4D0554A136823F0F80361696E
:1010B80043EAC103136011E00022514B1A6000F0AB
:1010C800B7FF054605E000F0B3FF401B022800F219
:1010D80021814A4B1B6813F0020FF4D1236813F0E7
:1010E800080F29D0A369ABB10122464B1A6000F062
:1010F8009FFF054605E000F09BFF401B022800F219
:101108000B813E4B5B6A13F0020FF4D00120FFF70E
:1011180007FF11E000223B4B1A6000F089FF0546EB
:1011280005E000F085FF401B022800F2F780334BF2
:101138005B6A13F0020FF4D1236813F0040F00F078
:1011480089802E4BDB6913F0805F0BD12B4BDA695A
:1011580042F08052DA61DB6903F080530193019B0E
:10116800012500E00025284B1B6813F4807F13D16C
:10117800254A136843F48073136000F059FF06464C
:1011880005E000F055FF801B642800F2C9801E4B63
:101198001B6813F4807FF4D0E368012B05D1174A4C
:1011A800136A43F00103136222E063B903F1804339
:1011B80003F504331A6A22F001021A621A6A22F04D
:1011C80004021A6214E0052B09D10C4B1A6A42F08A
:1011D80004021A621A6A42F001021A6208E0074B16
:1011E8001A6A22F001021A621A6A22F004021A62CA
:1011F800E368CBB100F01CFF06460FE00010024088
:1012080000004242800442420070004000F010FF9B
:10121800801B41F28833984200F28480494B1B6A54
:1012280013F0020FF2D00FE000F002FF064606E0CE
:1012380000F0FEFE801B41F28833984274D8414B7F
:101248001B6A13F0020FF3D125B13E4AD36923F08C
:101258008053D361E369002B68D03A4A526802F0A0
:101268000C02082A64D0022B37D10022364B1A60B0
:1012780000F0DEFE054604E000F0DAFE401B02281E
:1012880058D8304B1B6813F0007FF5D1236AB3F5AB
:10129800803F06D12B494B6823F40032A3681343DF
:1012A8004B602848436823F47411236A626A134325
:1012B8000B4343600122244B1A6000F0B9FE044638
:1012C80004E000F0B5FE001B022835D81D4B1B6852
:1012D80013F0007FF5D0002031E000221A4B1A608D
:1012E80000F0A6FE044604E000F0A2FE001B02285F
:1012F80024D8144B1B6813F0007FF5D100201EE0A2
:1013080001201CE003201AE0032018E0012016E069
:10131800032014E0032012E0032010E003200EE075
:1013280003200CE003200AE0032008E0002006E088
:10133800012004E0032002E0032000E0032002B0C3
:1013480070BD00BF001002406000424230B486B059
:10135800164D02AC28686968AA68EB680FC42B8A26
:10136800ADF80430124B5A6802F00C03082B19D15F
:10137800C2F3834306A90B4413F8103C12F4803FD0
:101388000CD00B4A5268C2F340420A4412F8140CBB
:10139800084AB2FBF0F003FB00F004E0064800FB4B
:1013A80003F000E0034806B030BC7047C84E0008A0
:1013B8000010024000127A0000093D0070B55C4B35
:1013C8001B6803F007038B420BD2594A136823F0BA
:1013D80007030B431360136803F007038B4240F0C5
:1013E8009780036813F0020F06D0524C636823F00D
:1013F800F0028368134363600D460446036813F0E4
:10140800010F4DD04268012A05D14A4B1B6813F4DD
:10141800003F0DD17EE0022A05D1464B1B6813F030
:10142800007F05D178E0434B1B6813F0020F75D09D
:1014380040494B6823F0030313434B6000F0F8FD69
:1014480006466368012B0ED106E000F0F1FD801B13
:1014580041F28833984263D8364B5B6803F00C033B
:10146800042BF2D11CE0022B15D106E000F0E0FDC0
:10147800801B41F28833984254D82E4B5B6803F0A6
:101488000C03082BF2D10BE000F0D2FD801B41F2D7
:101498008833984248D8274B5B6813F00C0FF3D178
:1014A800234B1B6803F00703AB420AD9204A136891
:1014B80023F007032B431360136803F00703AB42C1
:1014C80034D1236813F0040F06D01A494B6823F46B
:1014D800E062E36813434B60236813F0080F07D0FA
:1014E800144A536823F46053216943EAC1035360E3
:1014F800FFF72CFF0F4B5B68C3F303130E4AD35C53
:10150800D8400E4B1860002000F062FD002070BD2E
:10151800012070BD012070BD012070BD012070BD8B
:10152800032070BD032070BD032070BD012070BD75
:101538000020024000100240DC4E0008000000209D
:10154800014B1868704700BF0000002008B5FFF77E
:10155800F7FF044B5B68C3F30223034AD35CD8400C
:1015680008BD00BF00100240EC4E000808B5FFF7A8
:10157800E7FF044B5B68C3F3C223034AD35CD8403C
:1015880008BD00BF00100240EC4E000830B4036AEA
:1015980023F001030362036A4468826922F073023C
:1015A8000D682A4323F002038D682B43104DA8428F
:1015B80003D005F50065A84205D123F00803CD68DE
:1015C8002B4323F004030A4DA84203D005F5006518
:1015D800A84205D124F440744D692C438D692C43ED
:1015E800446082614A684263036230BC704700BF4E
:1015F800002C014030B4036A23F480730362036A49
:101608004468C26922F073020D682A4323F4007308
:101618008D6843EA0523124DA84203D005F50065FD
:10162800A84206D123F40063CD6843EA052323F4D6
:1016380080630B4DA84203D005F50065A84207D189
:1016480024F440544D6944EA05148D6944EA0514AC
:101658004460C2614A68C263036230BC704700BF1D
:10166800002C014030B4036A23F480530362036AF8
:101678004468C26922F4E6420D6842EA052223F46E
:1016880000538D6843EA0533094DA84203D005F598
:101698000065A84204D124F480444D6944EA8514C5
:1016A8004460C2614A680264036230BC704700BF8C
:1016B800002C014010B4036A046A24F00104046297
:1016C800846924F0F00444EA021223F00A0319435F
:1016D800826101625DF8044B704700BF10B4036A71
:1016E80023F0100303628469036A24F4704444EA13
:1016F800023223F0A00343EA0111826101625DF81E
:10170800044B704710B4846824F47F4442EA0323EE
:1017180019430C4384605DF8044B704710B50C46C0
:101728000268936823F0700349680B4323F00703AA
:1017380021680B4393606368502B1FD002D8402B5D
:101748000BD010BD602B1FD0702B22D10068E16830
:10175800A2682369FFF7D6FF10BD0368196A1A6AE1
:1017680022F001021A620268936923F0F0032469E7
:1017780043EA041393610368196210BD0068A16805
:101788002269FFF797FF10BD0068A1682269FFF77B
:10179800A5FF10BD704700BF38B590F83C30012B4D
:1017A80018D00446012580F83C50022380F83D30CB
:1017B800FFF7B4FF2268D36823F04003D3602268A0
:1017C800D36823F48043D36084F83D50002084F824
:1017D8003C0038BD022038BD0368244A904212D02C
:1017E80002F5006290420ED0B0F1804F0BD0A2F506
:1017F8009832904207D002F58062904203D002F5F9
:101808008062904203D123F070034A681343174A59
:10181800904212D002F5006290420ED0B0F1804F93
:101828000BD0A2F59832904207D002F58062904220
:1018380003D002F58062904203D123F44073CA6852
:10184800134323F080034A69134303608B68C36220
:101858000B688362054B984203D003F500639842F6
:1018680001D10B690363012343617047002C0140D8
:10187800C0B110B5044690F83D3013F0FF0F04D105
:10188800002380F83C30FFF785FF022384F83D30C1
:10189800214651F8040BFFF79FFF012384F83D30E0
:1018A800002010BD0120704730B4036A23F01003F4
:1018B8000362036A4468826922F4E6420D6842EAD8
:1018C800052223F020038D6843EA0513114DA84231
:1018D80003D005F50065A84206D123F08003CD6842
:1018E80043EA051323F040030A4DA84203D005F547
:1018F8000065A84207D124F440644D6944EA850490
:101908008D6944EA8504446082614A68826303629F
:1019180030BC7047002C014038B590F83C30012BA2
:1019280066D00D460446012380F83C30022380F837
:101938003D300C2A55D8DFE802F0075454541A54A5
:1019480054542E54545441000068FFF71FFE226877
:10195800936943F0080393612268936923F00403B1
:101968009361226891692B690B43936139E00068A0
:10197800FFF79AFF2268936943F400639361226832
:10198800936923F48063936122689369296943EA20
:101998000123936125E00068FFF72CFE2268D369D4
:1019A80043F00803D3612268D36923F00403D361A9
:1019B8002268D1692B690B43D36112E00068FFF7F5
:1019C80051FE2268D36943F40063D3612268D36966
:1019D80023F48063D3612268D369296943EA012328
:1019E800D361012384F83D30002084F83C0038BDE1
:1019F800022038BD10B401238B40046A24EA030393
:101A08000362036A8A401A4302625DF8044B704716
:101A180010B5044600680122FFF7ECFF23680C4A62
:101A2800934205D002F50062934203D1012202E0FD
:101A3800012200E000221AB15A6C42F400425A64B2
:101A48002268136843F001031360002010BD00BF33
:101A5800002C014010B404238B40046A24EA0303D9
:101A68000362036A8A401A4302625DF8044B7047B6
:101A780010B5044600680422FFF7ECFF2268536C97
:101A880043F4004353642268136843F0010313606E
:101A9800002010BD90F83C30012B22D0012380F8A3
:101AA8003C30CB6823F440728B68134323F4806284
:101AB8004B68134323F400620B68134323F48052EA
:101AC8000B69134323F400524B6913438A6923F4C7
:101AD8004043134302685364002380F83C3018469F
:101AE80070470220704700BF90F83C30012B21D08E
:101AF80030B4012280F83C20022380F83D3004688D
:101B0800636823F070036360046865680B682B439F
:101B180063600468A36823F08003A3600468A56871
:101B28004B682B43A36080F83D20002380F83C30AD
:101B3800184601E00220704730BC704790F8243006
:101B4800012B27D0012380F8243003689A6812F00B
:101B5800010F10D1124A926812F0010F0BD1114AED
:101B6800934208D110B45A6822F470240A682243B8
:101B78005A60002309E0836A43F02003836201234B
:101B8800002280F8242018467047002280F824207C
:101B9800184601E0022070475DF8044B704700BF0B
:101BA800002801400024014000F00700064AD368DD
:101BB80023F4E0631B041B0C43EA002040F0BF60E1
:101BC80040F40030D060704700ED00E030B4164BB0
:101BD800DC68C4F30224C4F10705042D28BF0425DA
:101BE800231D062B01D9033C00E00024012303FA3E
:101BF80005F5013D2940A140A340013B1A400A4395
:101C0800002806DA00F00F001201D2B2074B1A546E
:101C180007E01201D2B200F1604000F5614080F89F
:101C2800002330BC704700BF00ED00E014ED00E079
:101C3800410900F01F0001238340024A42F8213085
:101C4800704700BF00E100E00138B0F1807F0AD2A0
:101C5800064B5860F021064A82F82310002098604D
:101C680007221A6070470120704700BF10E000E0AB
:101C780000ED00E0042805D1054A136843F0040389
:101C880013607047024A136823F004031360704717
:101C980010E000E0704700BF08B5FFF7FBFF08BD84
:101CA800F0B583B000273C46E2E00122A2400B6871
:101CB8001340934240F0DB804D68122D2DD00BD895
:101CC800022D27D003D85DB3012D1ED035E0032D9A
:101CD80030D0112D1BD030E0684EB54220D008D846
:101CE800A6F58016B5421BD006F58036B54224D13C
:101CF80016E0634EB54213D006F58036B5420FD0D4
:101D0800A6F58016B54218D10AE0CF6815E0CF686D
:101D1800043712E0CF6808370FE0CF680C370CE0C3
:101D28008D684DB1012D02D10261082705E042619D
:101D3800082702E0002700E00427FF2B01D884468B
:101D480001E000F1040CFF2B02D84FEA840E03E0F7
:101D5800A4F1080E4FEA8E0EDCF800600F2202FA9A
:101D68000EF226EA020507FA0EF22A43CCF8002002
:101D78004A6812F0805F7AD0424A956945F00105B9
:101D88009561926902F001020192019AA208961CDB
:101D98003D4D55F8266004F0030E4FEA8E0E0F25D0
:101DA80005FA0EF526EA0506384DA8421FD005F5B6
:101DB8008065A84219D005F58065A84213D005F5BD
:101DC8008065A8420DD005F58065A84207D005F5C5
:101DD8008065A84201D105250AE0062508E004250A
:101DE80006E0032504E0022502E0012500E00025C5
:101DF80005FA0EF535430232234E46F822504A685A
:101E080012F4803F04D0224D2A681A432A6004E065
:101E18001F4D2A6822EA03022A604A6812F4003F2A
:101E280004D01B4D6A681A436A6004E0184D6A685A
:101E380022EA03026A604A6812F4801F04D0144D33
:101E4800AA681A43AA6004E0114DAA6822EA0302AC
:101E5800AA604A6812F4001F04D00D4DEA681343C3
:101E6800EB6004E00A4DEA6822EA0303EB60013400
:101E78000F2C7FF61AAF03B0F0BD00BF0000211091
:101E8800000031100010024000000140000801402D
:101E98000004014083680B4201D0012070470020F4
:101EA800704700BF0AB101617047090401617047BA
:101EB800C3685940C160704770B582B00446036872
:101EC80013F0010F5CD03E4BDB6913F0805F0BD140
:101ED8003B4BDA6942F08052DA61DB6903F08053E8
:101EE8000193019B012600E00026364B1B6813F482
:101EF800807F12D1334A136843F48073136000F073
:101F080097F8054604E000F093F8401B64284FD882
:101F18002C4B1B6813F4807FF5D0294B1B6A13F4F4
:101F2800407321D0626802F440729A421CD0244A5D
:101F3800136A23F44070244901250D6000250D60C3
:101F4800106213F0010F0FD000F072F8054606E09A
:101F580000F06EF8401B41F2883398422AD8184B9B
:101F68001B6A13F0020FF3D015490B6A23F4407271
:101F7800636813430B621EB1CB6923F08053CB61B6
:101F8800236813F0020F06D00D494B6823F4404232
:101F9800A36813434B60236813F0100F0CD0084953
:101FA8004B6823F48002636913434B60002004E00C
:101FB800032002E0032000E0002002B070BD00BF53
:101FC800001002400070004040044242704700BFC9
:101FD80010B50446074B1B680748A0FB033080096F
:101FE800FFF732FE4FF0FF3021460022FFF7EEFDEB
:101FF800002010BD00000020D34D621008B5074A2C
:10200800136843F0100313600320FFF7CDFD002091
:10201800FFF7DEFFFFF7DAFF002008BD00200240CF
:10202800024A136801331360704700BFE8000020BC
:10203800014B1868704700BFE800002030B583B036
:102048000190FFF7F5FF0546019CB4F1FF3F00D072
:102058000134FFF7EDFF401BA042FAD303B030BDB7
:10206800704700BF70B483B00023019390F8243008
:10207800012B00F08380012380F824304B68062B65
:102088000DD80668756B03EB8303053B1F229A4046
:1020980025EA02040A689A40224372631CE00C2B6A
:1020A8000DD80668356B03EB8303233B1F229A4048
:1020B80025EA02040A689A40224332630CE0066863
:1020C800F56A03EB8303413B1F229A4025EA020489
:1020D8000A689A402243F2620B68092B0DD90668F8
:1020E800F56803EB43031E3B07229A4025EA0204E6
:1020F8008A689A402243F2600BE00668356903EB70
:10210800430307229A4025EA02048A689A40224338
:1021180032610B68103B012B26D80368194A934299
:102128001CD19A6812F4000F20D19A6842F4000278
:102138009A600B68102B1BD1134B1B68134AA2FB28
:1021480003239B0C03EB83035B00019302E0019BD9
:10215800013B0193019B002BF9D10AE0836A43F00C
:1021680020038362012304E0002302E0002300E04F
:102178000023002280F82420184600E0022003B043
:1021880070BC7047002401400000002083DE1B4320
:1021980030B583B00023019303689A6812F0010FE9
:1021A8002FD19A6842F001029A60174B1B68174AB0
:1021B800A2FB03239B0C019302E0019B013B0193CB
:1021C800019B002BF9D10446FFF732FF054611E0C9
:1021D800FFF72EFF401B02280CD9A36A43F0100317
:1021E800A362E36A43F00103E362002384F8243026
:1021F800012007E023689B6813F0010FE8D0002056
:1022080000E0002003B030BD0000002083DE1B4347
:1022180090F82430012B70D010B50446012380F8C3
:102228002430FFF7B5FF0346002861D1A26A22F4E3
:10223800407222F0010242F48072A26222683049A0
:102248008A4205D1A1F58061496811F4702F0ED139
:10225800A16A21F48011A162516811F4806F1CD029
:10226800A16A21F4405141F48051A16215E0A16AAC
:1022780041F48011A16223498A4203D001F58061AB
:102288008A420AD11F49496811F4806F05D0A16AB2
:1022980021F4405141F48051A162A16A11F4805F98
:1022A80004D0E16A21F00601E16201E00021E16267
:1022B800002184F824106FF00201116022689168EF
:1022C80001F46021B1F5602F0DD10D498A4205D185
:1022D800A1F58061496811F4702F04D1916841F427
:1022E800A001916007E0916841F48011916002E0DB
:1022F800002284F82420184610BD0220704700BF31
:10230800002801400024014038B503689A6812F09B
:10231800010F1ED004469A6822F001029A60FFF766
:1023280087FE05460EE0FFF783FE401B022809D909
:10233800A36A43F01003A362E36A43F00103E36274
:10234800012038BD23689B6813F0010FEBD10020F2
:1023580038BD002038BD00BF002800F0888070B567
:102368000446836A23B9C36280F82430FFF778FEF5
:102378002046FFF7C9FFA36A13F0100F71D1002898
:102388006FD1A36A23F4885323F0020343F00203B6
:10239800A36262682168374B994206D1E369B3F5B5
:1023A800402F03D14FF4002300E0E3691343E568AD
:1023B80043EA4503A268B2F5807F04D0012A05D11B
:1023C8004FF4807203E04FF4807200E000226669E7
:1023D800012E0FD135B9A569013D42EA453242F4D3
:1023E800006207E0A56A45F02005A562E56A45F0A8
:1023F8000105E5624D6825F469452A434A6021686C
:102408008D681D4A2A401A438A60A268B2F5807F07
:1024180001D0012A03D12269013A110500E0002107
:102428002568EA6A22F470020A43EA62226891681F
:10243800124A0A40934208D10023E362A36A23F0B8
:10244800030343F00103A36270BDA36A23F01203E0
:1024580043F01003A362E36A43F00103E36201203F
:1024680070BDA36A43F01003A362012070BD012070
:10247800704700BF003C0140FDF7E1FFFE0E1FFF63
:102488002DE9F843814601680B6923F44052C3687B
:1024980013430B6181680369194343691943006851
:1024A800C26822F4B05323F00C030B43C360D9F87D
:1024B80000104B6923F44072D9F8183013434B616C
:1024C800D9F800505B4B9D4259D1FFF74FF800EB0C
:1024D800800000EB8000D9F80440A400B0FBF4F4BD
:1024E800554EA6FB043464092401FFF73FF800EBBE
:1024F800800000EB8000D9F804309B00B0FBF3F7B4
:10250800FFF734F800EB800000EB8000D9F80430C6
:102518009B00B0FBF3F3A6FB03235B094FF06408B1
:1025280008FB13731B013233A6FB03235B0903F07B
:10253800F0031C44FFF71AF800EB800000EB800062
:10254800D9F804309B00B0FBF3F7FFF70FF800EB66
:10255800800000EB8000D9F804309B00B0FBF3F357
:10256800A6FB03235B0908FB13731B013233A6FB8D
:102578000323C3F343131C44AC60BDE8F883FEF7A0
:10258800E5FF00EB800000EB8000D9F80440A400D0
:10259800B0FBF4F4284EA6FB043464092401FEF7CA
:1025A800D5FF00EB800000EB8000D9F804309B00D9
:1025B800B0FBF3F7FEF7CAFF00EB800000EB8000EA
:1025C800D9F804309B00B0FBF3F3A6FB03235B09A7
:1025D8004FF0640808FB13731B013233A6FB032377
:1025E8005B0903F0F0031C44FEF7B0FF00EB80002A
:1025F80000EB8000D9F804309B00B0FBF3F7FEF73E
:10260800A5FF00EB800000EB8000D9F804309B00A8
:10261800B0FBF3F3A6FB03235B0908FB13731B0151
:102628003233A6FB0323C3F343131C44AC60BDE859
:10263800F88300BF003801401F85EB51704700BF89
:1026480068B310B5044690F8393013F0FF0F04D181
:10265800002380F83830FFF7F1FF242384F839305D
:102668002268D36823F40053D3602046FFF708FF9D
:102678002268136923F4904313612268536923F095
:102688002A0353612268D36843F40053D3600020BF
:10269800E063202384F8393084F83A3010BD0120F3
:1026A800704700BF03685A6912F4806F0DD06FF449
:1026B80080625A610423036400230363202280F8A4
:1026C8003D2080F83C30012070470020704700BF53
:1026D800F8B506460C4617461D4614E0B5F1FF3F0F
:1026E80011D02DB1FFF7A4FC069BC01AA8420AD945
:1026F80000233363202286F83D2086F83E3086F892
:102708003C300320F8BDC4F30743012B08D13368DC
:102718005B6924EA03039BB2B3FA83F35B0907E01E
:1027280033689B6924EA03039BB2B3FA83F35B091A
:10273800BB42D3D00020F8BDF8B504460D46164676
:102748001F4629E023685A6912F4806F12D01A686C
:1027580042F400721A6023686FF480625A6104239D
:10276800236400232363202284F83D2084F83C302E
:102778000120F8BDB6F1FF3F0ED026B1FFF758FC97
:10278800C01BB04208D900232363202284F83D20CF
:1027980084F83C300320F8BDC5F30743012B08D16A
:1027A80023685B6925EA03039BB2003318BF012342
:1027B80007E023689B6925EA03039BB2003318BF2F
:1027C8000123002BBED10020F8BD00BFF0B583B0B7
:1027D80004460F4616461D46C36A042B04D0012B37
:1027E80002D013F5803F05D12268136843F4807343
:1027F800136007E0036B122B04D10268136843F4DB
:1028080080731360009520464FF001110022334673
:10281800FFF75EFF58BB2369B3F5804F04D12368E7
:1028280007F0FE071F6115E0226807F44073DB110B
:1028380043F0F00313612046114932462B46FFF757
:102848007BFF20B1236C042B13D1012314E02368F0
:10285800FFB21F6120460B4932462B46FFF76CFF3B
:10286800034648B1236C042B05D1012304E003235C
:1028780002E0032300E00323184603B0F0BD00BFC5
:1028880008000100020001002DE9F04184B004466F
:102898000F4616461D46C26A01680B6843F48063FA
:1028A8000B60042A04D0012A02D012F5803F05D11A
:1028B8002268136843F48073136007E0036B112BDD
:1028C80004D10268136843F48073136000952046AE
:1028D8004FF0011100223346FFF7FAFE002851D1CC
:1028E8002369B3F5804F05D1236847F00107FFB28C
:1028F8001F613AE0236807F440784FEAD81848F097
:10290800F0021A612046264932462B46FFF714FF8B
:1029180020B1236C042B37D101233CE02368FFB29C
:102928001F6120461F4932462B46FFF705FF20B19D
:10293800236C042B2AD101232DE000220392236863
:1029480059690391996903910399196841F4807150
:102958001960009520464FF001113346FFF7B8FE85
:10296800B0B9226848F0F103136120460D49324698
:102978002B46FFF7E1FE034668B1236C042B09D10F
:10298800012308E0032306E0032304E0032302E015
:10299800032300E00323184604B0BDE8F08100BF1C
:1029A800080001000200010070B504460D461646F5
:1029B80019E02046FFF776FEE0B9B5F1FF3F12D0E7
:1029C80025B1FFF735FB801BA8420CD9236C43F0D7
:1029D8002003236400232363202284F83D2084F805
:1029E8003C30032070BD23685B6913F0800FE0D092
:1029F800002070BD012070BD70B504460D46164616
:102A080019E02046FFF74EFEE0B9B5F1FF3F12D0BE
:102A180025B1FFF70DFB801BA8420CD9236C43F0AE
:102A28002003236400232363202284F83D2084F8B4
:102A38003C30032070BD23685B6913F0040FE0D0BD
:102A4800002070BD012070BD70B505460C461646C5
:102A580022E05A6912F0100F0CD06FF010025A6180
:102A680000232B642B63202285F83D2085F83C3019
:102A7800012070BD24B1FFF7DBFA801BA0420BD9FF
:102A88002B6C43F020032B64202385F83D30002372
:102A980085F83C30032070BD2B685A6912F0400F4E
:102AA800D7D0002070BD00BF704700BF002800F0DD
:102AB800838038B5044690F83D3013F0FF0F04D1F9
:102AC800002380F83C30FFF7EFFF242384F83D30E3
:102AD8002268136823F001031360FEF737FD374BB4
:102AE800A3FB00239B0C2268536021686568344A65
:102AF800954201D8013308E04FF4967202FB03F3C4
:102B0800304AA2FB03239B0901330B6221686368E7
:102B18002B4A934208D85B00B0FBF3F0C0F30B03D9
:102B2800032B2BD8042029E0A5684DB903EB4302F9
:102B3800B0FBF2F2C2F30B02B2FA82F252090AE0D7
:102B480003EB830202EB8202B0FBF2F2C2F30B0248
:102B5800B2FA82F2520982B935B903EB4303B0FBEA
:102B6800F3F040F4004009E003EB830303EB830335
:102B7800B0FBF3F040F4404000E00120C861226857
:102B8800E169236A0B43136022682169E3680B43F8
:102B9800936022686169A3690B43D3602268136854
:102BA80043F00103136000202064202384F83D30A3
:102BB800206384F83E0038BD0120704783DE1B4344
:102BC800A0860100D34D62102DE9F04184B004467F
:102BD8000D4690461F46FFF72BFA94F83D30DBB2BE
:102BE800202B40F0A0800646009020465449012240
:102BF8001923FFF76DFD002840F0978094F83C30CA
:102C0800012B00F09480012384F83C3023681A6873
:102C180012F0010F03D11A6842F001021A6022680B
:102C2800136823F400631360212384F83D301023D4
:102C380084F83E3000232364C4F824806785A3F514
:102C48008033E362638D2385204629460A9A3346FA
:102C5800FFF7BCFD054660B1236C042B04D10023AB
:102C680084F83C30012567E0002384F83C300325D4
:102C780062E00023039323685A6903929B690393D4
:102C8800039B3FE020460A993246FFF78DFE48B184
:102C9800236C042B4DD12268136843F4007313602E
:102CA800012549E02268636A591C61621B78136137
:102CB800638D013B9BB26385238D013B9BB22385CA
:102CC8002268516911F0040F0CD05BB1636A591C7A
:102CD80061621B781361638D013B9BB26385238D11
:102CE800013B238520460A993246FFF785FE48B105
:102CF800236C042B1FD12268136843F400731360FC
:102D0800012519E0238D002BBCD12268136843F4F8
:102D180000731360202384F83D30002384F83E308C
:102D280084F83C3008E0022506E0022504E002258C
:102D380002E0032500E00325284604B0BDE8F08141
:102D4800020010002DE9F04186B004460D46904679
:102D58001F46FFF76DF994F83D30DBB2202B40F0A9
:102D68005C81064600902046944901221923FFF70A
:102D7800AFFC002840F0538194F83C30012B00F060
:102D88005081012384F83C3023681A6812F0010F3F
:102D980003D11A6842F001021A602268136823F40A
:102DA80000631360222384F83D30102384F83E30FA
:102DB80000232364C4F824806785A3F58033E36285
:102DC800638D2385204629460C9A3346FFF75CFD20
:102DD800054660B1236C042B04D1002384F83C30F1
:102DE800012529E1002384F83C30032524E1238DC3
:102DF8005BB9029323685A6902929A690292029A0D
:102E08001A6842F400721A60FAE0012B13D12268A2
:102E1800136823F48063136072B600230393236856
:102E28005A6903929A690392039A1A6842F40072E3
:102E38001A6062B6E4E0022B13D12268136843F4E7
:102E48000063136072B60023049323685A690492DE
:102E58009A690492049A1A6822F480621A6062B627
:102E6800CEE02268136843F480631360002305935F
:102E780023685A6905929B690593059BC0E0032B5B
:102E880000F29180012B19D120460C993246FFF7A8
:102E9800DBFD28B1236C202B40F0C5800325CBE057
:102EA800636A5A1C6262226812691A70238D013B98
:102EB8002385638D013B9BB26385A1E0022B2BD157
:102EC800009620463E4900220C9BFFF701FC002893
:102ED80040F0AB8072B62268136843F40073136045
:102EE800636A5A1C6262226812691A70238D013B58
:102EF8002385638D013B9BB2638562B6636A5A1C66
:102F08006262226812691A70238D013B2385638DE2
:102F1800013B9BB2638573E0009620462849002256
:102F28000C9BFFF7D5FB002840F0818022681368CE
:102F380023F48063136072B6636A5A1C6262226863
:102F480012691A70238D013B2385638D013B9BB267
:102F58006385009620461A4900220C9BFFF7B8FBB0
:102F6800002866D12268136843F400731360636A0B
:102F78005A1C6262226812691A70238D013B2385EC
:102F8800638D013B9BB2638562B6636A5A1C6262B9
:102F9800226812691A70238D013B2385638D013BDA
:102FA8009BB263852CE020460C993246FFF74CFD16
:102FB80040B1236C202B3ED103253DE002001000D8
:102FC80004000100636A5A1C6262226812691A705E
:102FD800238D013B2385638D013B9BB26385236869
:102FE8005A6912F0040F0BD0626A511C61621B69A6
:102FF8001370238D013B2385638D013B9BB2638551
:10300800238D002B7FF43BAF202384F83D30002331
:1030180084F83E3084F83C300EE002250CE00225AE
:103028000AE0022508E0012506E0032504E003255F
:1030380002E0032500E00125284606B0BDE8F0813E
:1030480000283ED010B403460168204A91420AD8AD
:103058001F4A0A441F49A1FB021212099200026486
:103068001D4AC26309E01D4A0A441A49A1FB02121B
:103078001209920002641A4AC263022283F82120CC
:103088001C68226822F47F5222F03002586899683E
:103098000843D96808431969084359690843996975
:1030A8000843D96901430A43226000209862D86224
:1030B800186358639863012283F8212083F820005D
:1030C80001E0012070475DF8044B70470704024097
:1030D800F8FFFDBFCDCCCCCC00000240F8FBFDBF13
:1030E800000402400F4B1A6842F001021A60596846
:1030F8000D4A0A405A601A6822F0847222F480321B
:103108001A601A6822F480221A605A6822F4FE02B1
:103118005A604FF41F029A604FF00062034B9A60A6
:10312800704700BF001002400000FFF800ED00E00B
:1031380030B597B01F4BDA6942F40032DA61DA69C8
:1031480002F400320092009A5A6942F001025A6170
:103158005B6903F001030193019B174D06954FF43A
:10316800E13307930024089409940A9408230B93E5
:103178000C940D9406A8FFF763FA6B6943F080037B
:103188006B61042302930123049302230393032313
:1031980005930A4802A9FEF783FD094B1C60094AFA
:1031A8009A605C6090221A604FF0E062803B5A603F
:1031B80017B030BD00100240004400400008014034
:1031C80080000240044400402DE9F0418AB04A4D95
:1031D800EB6943F48003EB61EB6903F4800301932B
:1031E800019B6B6943F001036B616B6903F0010399
:1031F8000293029B0E2001210422FEF7E7FC0E2019
:10320800FEF716FD0F2001210322FEF7DFFC0F2039
:10321800FEF70EFD394E3A4B33603A4B736000248B
:10322800B460F4604FF4804333617461B461F46155
:1032380034623046FFF73AFC6B6943F001036B6177
:103248006B6903F001030393039BAB6943F0080325
:10325800AB61AB6903F008030493049B4FF440632C
:1032680006931223079301230893032309932648FF
:1032780006A9FEF715FDEB6943F48003EB61EB69E2
:1032880003F480030593059B204D214B2B606C6054
:10329800AC604FF08008C5F80C802C616C61AC61A3
:1032A8004FF48057EF612846FFF7CAFEB5636E6298
:1032B800184D194B2B6010236B60AC60C5F80C805F
:1032C8002C616C61AC61EF612846FFF7B9FE75634C
:1032D8006E62212021462246FEF778FC2120FEF767
:1032E800A7FC222021462246FEF770FC2220FEF78A
:1032F8009FFC0AB0BDE8F081001002401C010020CC
:1033080000580040A0860100000C0140B0010020D8
:1033180058000240F4010020440002402DE9F04F1B
:1033280089B07B4B9A6942F004029A619A6902F06B
:1033380004020192019A9A6942F008029A619A6914
:1033480002F008020292029A9A6942F010029A6107
:103358009B6903F010030393039B002305930693D3
:10336800022707974FF0200A0DEB0A0444F810AD26
:1033780068482146FEF794FC40230493654821469B
:10338800FEF78EFC8025049562482146FEF788FCEE
:103398004FF48063049360482146FEF781FC4FF4A4
:1033A800006304935C482146FEF77AFC4FF480568C
:1033B800049659482146FEF773FC0496574821465F
:1033C800FEF76EFC049755482146FEF769FC4FF05E
:1033D8000108CDF814804FF00409CDF810904D483D
:1033E8002146FEF75DFC102604964C482146FEF760
:1033F80057FCCDF810A049482146FEF751FC03239D
:103408000593CDF8108044482146FEF749FCCDF8D5
:10341800108042482146FEF743FC4FF0080BCDF8D8
:1034280010B03D482146FEF73BFC04973A48214638
:10343800FEF736FC049638482146FEF731FCCDF8F5
:1034480010A035482146FEF72BFCCDF810903248E5
:103458002146FEF725FCCDF810B030482146FEF78E
:103468001FFCCDF810902D482146FEF719FC059752
:103478004023049328482146FEF712FC0495264869
:103488002146FEF70DFC4FF48079CDF810902248C4
:103498002146FEF705FC049520482146FEF700FC6E
:1034A800CDF810801B482146FEF7FAFB049719480F
:1034B8002146FEF7F5FBCDF8109018482146FEF797
:1034C800EFFB4FF40073049314482146FEF7E8FB22
:1034D8004FF48063049311482146FEF7E1FB4FF453
:1034E800005304930B482146FEF7DAFB4FF4804360
:1034F800049308482146FEF7D3FB4FF40043049396
:1035080004482146FEF7CCFB09B0BDE8F08F00BFA8
:1035180000100240000C014000100140000801406A
:103528002DE9F04F99B0754B9A6942F400629A619F
:103538009A6902F400620192019A9A6942F400526F
:103548009A619B6903F400530293029B6C4EDFF867
:10355800B891C6F80090002474604FF02008C6F8AF
:1035680008804FF4FA6BC6F80CB034617461B4612A
:103578003046FEF77DF9102316931794304616A9A6
:10358800FEF7B2FA60230F9310941194082712974C
:10359800139414944FF40073159330460FA92246E0
:1035A800FEF7BAF930460FA90422FEF7B5F93046FE
:1035B8000FA93A46FEF7B0F94FF4006308934FF4A9
:1035C800806309930A94CDF82C800C940D940E9482
:1035D80030460DEB0801FEF75DFA4A4DDFF82CA1E5
:1035E800C5F800A06C60C5F80880C5F80CB02C615F
:1035F8006C61AC612846FEF73BF9CDF85880802312
:103608001793284616A9FEF76FFA049418A90523FC
:1036180041F8543D2846FEF7BFF860230F931094F5
:1036280011941297139414944FF400731593284629
:103638000FA92246FEF770F928460FA90422FEF7C3
:103648006BF928460FA93A46FEF766F94FF400636E
:1036580008934FF4806309930A94CDF82C800C9456
:103668000D940E9428460DEB0801FEF713FADAF8CC
:10367800443023F40043CAF84430D9F8443023F4E2
:103688000043C9F8443028462146FEF7C1F92846C8
:103698000421FEF7BDF928463946FEF7B9F9284650
:1036A8002146FEF7E5F928460421FEF7E1F9284608
:1036B8003946FEF7DDF930462146FEF7A9F93046CE
:1036C8000421FEF7A5F930463946FEF7A1F9304640
:1036D8002146FEF7CDF930460421FEF7C9F93046F8
:1036E8003946FEF7C5F92B6801221A633268136858
:1036F80043F00103136019B0BDE8F08F00100240D9
:10370800700100207C020020002C014000340140A0
:103718002DE9F04387B0414EB36943F40073B361B8
:10372800B36903F400730093009B3D4C3D4B236049
:103738004FF48073A3600025E56065614FF4402372
:10374800E36165604FF00508C4F810802046FEF775
:1037580003FE354A536843F48023536006A94FF4A7
:10376800C02341F8043D2046FEF7E8F901230493FD
:103778000E2202920393204602A9FEF773FC0295DB
:1037880002270397204602A9FEF76CFC04970B2733
:10379800029703230393204602A9FEF763FC4FF028
:1037A8000C09CDF8089004230393204602A9FEF7DC
:1037B80059FCCDF80890CDF80C80204602A9FEF7F8
:1037C80051FC23689A6842F480729A609A6842F0C1
:1037D80001029A60736943F001037361736903F02E
:1037E80001030193019B114B1D60C3F80480104A2B
:1037F8009A60104ADA6040F6A2221A601A6842F00B
:1038080001021A60384629462A46FEF7DFF938468B
:10381800FEF70EFA07B0BDE8F08300BF00100240C3
:103828003802002000240140000001400800024046
:103838004C24014068020020F0B585B0274B9A69F6
:1038480042F480629A619B6903F480630093009B51
:10385800234C244B23604FF48073A3600023E36060
:1038680063614FF46022E2616360052626612046A9
:10387800FEF772FD012303930F2201920293204663
:1038880001A9FEF7EFFB0D230193022502952046BF
:1038980001A9FEF7E7FB03950A2301930327029783
:1038A800204601A9FEF7DEFB01950423029320467A
:1038B8000DEB0301FEF7D6FB01970296204601A9FE
:1038C800FEF7D0FB23689A6842F480729A609A687F
:1038D80042F001029A6005B0F0BD00BF001002403E
:1038E800EC0000200028014000B583B0084A4023BE
:1038F800137000235370642300930648A421022305
:10390800FFF762F90A20FEF799FB03B05DF804FBA4
:10391800BC0200201C010020F0B583B0114D00242A
:103928002C70114E642700973046A4212A460123A3
:10393800FFF74AF90220FEF781FB00973046A421E1
:103948002A460623FFF7FEF9224607E0054B9B5C53
:1039580083F01703173305498B540132052AF5DD27
:1039680003B0F0BDBC0200201C010020A400002010
:1039780030B597B002250C950123109310231193AD
:103988001395002414944FF4601315930CA8FDF7B5
:10399800DDFA0F230793089509944FF480630A937F
:1039A8000B9407A82946FDF709FD01954FF44043FC
:1039B800039301A8FEF780FAFDF7C2FD084BA3FBAD
:1039C80000308009FEF740F90420FEF753F94FF064
:1039D800FF3021462246FEF7F9F817B030BD00BF88
:1039E800D34D6210000000002DE9F04F85B0FEF7BE
:1039F80005FBC14CA36943F00103A361A36903F06C
:103A080001030393039B0320FEF7CEF86FF00B002E
:103A180000210A46FEF7DAF86FF00A0000210A468C
:103A2800FEF7D4F86FF0090000210A46FEF7CEF839
:103A38006FF0040000210A46FEF7C8F86FF0030093
:103A480000210A46FEF7C2F86FF0010000210A467D
:103A5800FEF7BCF84FF0FF3000210A46FEF7B6F833
:103A6800FFF786FF636923F001036361FFF756FCE4
:103A7800FFF756FDFFF74CFEFFF7DEFEFFF758FB9A
:103A88009E4820210122FEF70DFA9D48FEF7C0FB53
:103A98009C48FEF7BDFB082405E09B4B1C70642086
:103AA800FEF7CCFA013C002CF7DA0024964B1C7088
:103AB800964804210122FEF7F5F9FFF785FBFFF789
:103AC80013FF0122924B1A70A24601E0AA4634461F
:103AD8000220FEF7B3FAFFF71FFF8E4B1B78A3F106
:103AE8007F0505EB85035B00B3F57A7F04DC8A4D1F
:103AF8009D42B8BF1D4601E04FF47A75874B1D60A3
:103B0800844B5B78A3F17F0707EB87035B00B3F572
:103B18007A7F04DC804F9F42B8BF1F4601E04FF414
:103B28007A777F4B1F604FF0000B7E4BC3F800B0D5
:103B38007D4E3068FCF7F8FC69A3D3E90023FCF755
:103B480059FD804689462846FCF7EEFC66A3D3E972
:103B58000023FCF74FFD02460B4640464946FCF75A
:103B680097FBFCF7E1FF80463060704D2868FCF752
:103B7800DBFC5BA3D3E90023FCF73CFDCDE90001A6
:103B88003846FCF7D1FC58A3D3E90023FCF732FDF3
:103B980002460B46DDE90001FCF77AFBFCF7C4FF9F
:103BA80028605846414600F0B1FC0120296800F021
:103BB800ADFC3068FCF7B8FC00225D4BFCF71AFD41
:103BC80006460F462868FCF7AFFC0022584BFCF766
:103BD80011FD804689463046394642464B46FCF739
:103BE80055FBCDE900010022524BFCF793FF78B951
:103BF800DDE900013EA3D3E90023FCF76DFF28B9F6
:103C0800DDE90001FCF790FF054603E0424D01E0C5
:103C18004FF47A753046394642464B46FCF738FB36
:103C280006460F460022434BFCF774FF78B930462E
:103C380039462FA3D3E90023FCF74EFF28B93046B5
:103C48003946FCF771FF064603E0334E01E04FF4B6
:103C58007A760220294600F059FC0320314600F00C
:103C680055FC04F132039E4212DA323CA6420FDDC3
:103C78000AF132039D420BDAAAF1320A554507DDF3
:103C8800284B1B68312B03D82B4B1D602B4B1E6018
:103C980000F042FC0022234B1A6018480221FEF76C
:103CA800F9F800284ED00022194B1A701348022147
:103CB800FEF7F0F80028F9D10024134B1C70204BB4
:103CC8001C7005E0104B1C706420FEF7B7F9013436
:103CD800072CF7DD094820210022FEF7E3F8FEE76C
:103CE800CDCCCCCCCCCCEC3F9A9999999999B93F49
:103CF8000000000000408FC0001002400008014092
:103D080038020020EC000020CC000020000C01400C
:103D1800C4000020A400002018FCFFFF14030020AA
:103D280004030020040000201003002008030020E2
:103D38000000E03F00408F40D0000020C800002075
:103D4800B0000020214B1C6820462149FDF7C0F82F
:103D580058B120461F49FDF7D9F830B105221E4B4E
:103D68001A7008221D4B1A70B0E620461949FDF753
:103D7800AFF858B120461A49FDF7C8F830B1052206
:103D8800154B1A700122154B1A709FE620461449EC
:103D9800FDF79EF898B10024104B1C70114B1C7055
:103DA80005E00D4B1C706420FEF748F90134072C20
:103DB800F7DD0D4820210022FEF774F8FEE7002306
:103DC800054A1370054A137080E600BF18000020EA
:103DD8000000104200000442CC000020B000002087
:103DE8000000F041C400002000080140000000006D
:103DF8000222854B5A60854B1B68B3F57A7F3ADA05
:103E08000133824A1360824A938899B281480368D1
:103E18000B4403EBD3735B100360D38899B27E48DD
:103E280003680B4403EBD3735B100360138899B2E8
:103E38007A4803680B4403EBD3735B100360538821
:103E480099B2774803680B4403EBD3735B100360A4
:103E5800538999B2734803680B4403EBD3735B101F
:103E6800036013899AB270490B68134403EBD37348
:103E78005B100B6070472DE9F0416C4B1C886C4B54
:103E8800A3FB04235B09642202FB13439BB223BBFD
:103E9800684D2868FCF75AFB53A3D3E90023FCF7C5
:103EA800A9FB06460F465A4B988980B2FCF76AFF71
:103EB800FCF74CFB4EA3D3E90023FCF79BFB4EA376
:103EC800D3E90023FCF796FB02460B4630463946F9
:103ED800FCF7DEF9FCF750FE28604D4B588980B29C
:103EE800504B1D68401BFCF71FFB45A3D3E900237B
:103EF800FCF780FB00220023FCF7EEFD80B1444B69
:103F0800588980B2401BFCF70FFB3DA3D3E900237F
:103F1800FCF770FB0022484BFCF7DEFDB8B90FE058
:103F28003B4B588980B2401BFCF7FEFA34A3D3E917
:103F38000023FCF75FFB0022404BFCF7EBFD30B998
:103F48003F4B1B68322B02D83E4B1B782BB93E4A9D
:103F5800536C23F40043536404E03B4A536C43F42A
:103F6800004353642A4B188980B22F4B1D68401BAD
:103F7800FCF7DAFA22A3D3E90023FCF73BFB002283
:103F88000023FCF7A9FD80B1214B188980B2401BA2
:103F9800FCF7CAFA1AA3D3E90023FCF72BFB00228B
:103FA800254BFCF799FDC0B90FE0194B188980B271
:103FB800401BFCF7B9FA12A3D3E90023FCF71AFB5C
:103FC80000221E4BFCF7A6FD38B91D4B1B68322B8F
:103FD80003D81C4B1B78002B3AD11C4A536C23F492
:103FE8000043536439E000BF2B8716D9CEF7EF3F63
:103FF800F5E4E827181C9B3FFCA9F1D24D62503F1D
:104008007B14AE47E17A943F00000240AC000020E8
:10401800680200200C000020080000201400002086
:10402800100000201C00002020000020D4000020E8
:104038001F85EB5118000020008041C000804140DE
:1040480004000020C400002000340140002C01407E
:10405800914A536C43F40043536490498B6813F0BE
:10406800200F0CBF012200228B6813F0400F0CBFF9
:1040780001230023896811F0800F0CBF012500255A
:104088008749886810F4806F0CBF012000208E6873
:1040980016F4006F0CBF01270027896811F4805FB0
:1040A80003EB450302EB43037E4EF35C7E490B6052
:1040B8000B6803F102030B600D687C4B83FB05E280
:1040C800A2EBE57202EB42024FEA4202A5EB0202C2
:1040D8000A600CBF022200223A4400EB4202B05CA4
:1040E800734A1060106802301060106883FB005338
:1040F800A3EBE07303EB43035B00C31A1360096887
:104108006C4883889BB26C4A12689A1AC3889BB21F
:104118006A4800681B1A052918D8DFE801F0030768
:104128000A0D1013D31A664A136012E0644B1A6022
:104138000FE0634B1A600CE0614A136009E0604AC3
:10414800136006E09B1A5E4A136002E000225C4B93
:104158001A600134A4B25B4B1C805B4B1878A8B181
:104168005A4BA3FB04231B0B594A1278013293FBC9
:10417800F2F102FB11334BB994FBF0F300FB13444B
:104188004CB954481021FDF793FE04E05148102122
:104198000022FDF787FE504BD3F800E0424B1B6826
:1041A800052B22D8DFE803F003080E12161C74460C
:1041B800CEF1000E00251CE0CEF1000574464FF04C
:1041C800000E16E0CEF10005002412E0CEF1000446
:1041D80000250EE0CEF1000475464FF0000E08E011
:1041E8007546CEF1000E002403E04FF0000E744631
:1041F80075463A4B1E682E4B1B68052B1AD8DFE80C
:1042080003F003070B0E111532467642002114E025
:1042180071423246002610E0714200220DE07242DF
:1042280000210AE072423146002606E03146764215
:10423800002202E0002632463146274B1B68002B3D
:1042480050DD274B1868184B1F680537174B83FB41
:1042580007C3A3EBE77303EB43035B00FB1A052BD0
:104268006FD8DFE803F003070B0E1115074640422D
:1042780000236BE043420746002067E043420027E3
:1042880064E04742002361E04742034600205DE0C6
:1042980003464042002759E0002C0140000C014031
:1042A80000100140F44E0008B8000020ABAAAA2A6A
:1042B800C0000020680200200C0000200800002038
:1042C800D8000020D4000020CC0000205917B7D116
:1042D800B000002000080140C8000020D0000020E5
:1042E800B4000020814B18684742814B1B6803F1DA
:1042F800010C804B83FB0C83A3EBEC7303EB4303B0
:104308005B00C3EB0C03052B04D8DFE803F01E07A2
:104318000A0E131700200746034617E0034600203D
:1043280014E003463846002710E03B460746184687
:1043380000230BE03B460746002007E03B460027EA
:1043480004E000200746034600E000231D443C44E7
:104358007044694B1B68002B33DD684BD3F800E0D1
:10436800674B1F680537634B83FB07C3A3EBE773F2
:1043780003EB43035B00FB1A052B56D8DFE803F079
:1043880003080E12161C7746CEF1000E002352E0E9
:10439800CEF1000377464FF0000E4CE0CEF100035B
:1043A800002748E0CEF10007002344E0CEF10007E3
:1043B80073464FF0000E3EE07346CEF1000E002724
:1043C80039E04E4BD3F800E0CEF100074C4B1B68A8
:1043D80003F1010C474B83FB0C83A3EBEC7303EB5A
:1043E80043035B00C3EB0C03052B04D8DFE803F0A1
:1043F80022080C10151A4FF0000E774673461AE083
:1044080073464FF0000E16E07346BE46002712E0D2
:104418003B4677469E4600230DE03B4677464FF0E5
:10442800000E08E03B46002705E04FF0000E7746F7
:10443800734600E0002319443A440EEB060305F5E1
:104448007A7540F2C676B54203DC0A2DB8BF0A2554
:1044580001E040F2C6752B4E756304F57A7440F29C
:10446800C675AC4203DC0A2CB8BF0A2401E040F24E
:10447800C674244DAC6300F57A7040F2C674A0424D
:1044880003DC0A28B8BF0A2001E040F2C6701D4CC0
:10449800E06301F57A7140F2C670814203DC0A29B3
:1044A800B8BF0A2101E040F2C6711748416302F51E
:1044B8007A7240F2C6718A4203DC0A2AB8BF0A221D
:1044C80001E040F2C67210498A6303F57A7340F23C
:1044D800C672934203DC0A2BB8BF0A2301E040F2FC
:1044E800C673094AD363BDE8F08100BFB400002059
:1044F800B8000020ABAAAA2AD0000020BC000020E7
:10450800C000002000340140002C0140014B23F87A
:10451800101070477C03002030B583B0144C20463F
:104528000021642200F08EF812490A884B88888896
:10453800C98800B2009009B2019120460E4912B212
:104548001BB200F087F80D4B5B6873B90B4C2368FE
:1045580023F001032360064D284600F09FF86060B1
:10456800E560236843F00103236003B030BD00BF5A
:10457800180300207C030020FC4E00088000024045
:10458800704700BFFEE700BFFEE700BFFEE700BFC1
:10459800FEE700BF704700BF704700BF704700BF0D
:1045A80008B5FDF73DFDFDF777FB08BD002103E0E9
:1045B8000B4B5B58435004310A480B4B42189A4244
:1045C800F6D30A4A02E0002342F8043B084B9A4219
:1045D800F9D3FEF787FD00F00FF8FFF705FA7047EB
:1045E8004C4F0008000000208800002088000020B0
:1045F800D0030020FEE700000E4B70B51E460E4C9F
:104608000025E41AA410A54204D056F8253098478E
:104618000135F8E700F048FC084B094C1E46E41A3F
:10462800A4100025A54204D056F825309847013536
:10463800F8E770BD444F0008444F0008444F000895
:10464800484F000803460244934202D003F8011B76
:10465800FAE770470EB400B54FF402719CB0ADF89C
:1046680014106FF00041049107914FF6FF711DABD4
:10467800ADF81610084953F8042B02900690086804
:1046880002A9019300F06CF8029B00221A701CB07A
:104698005DF804EB03B0704784000020034613F86C
:1046A800012B002AFBD1181A013870472DE9F04771
:1046B8008E688246B3420C469046994640D38A8912
:1046C80012F4906F3AD02568096902236F1A656958
:1046D80005EB450595FBF3F57B1C4B449D4238BF24
:1046E8001D4653050FD5294600F03AFB064698B1FA
:1046F80021693A4600F0CAFAA38923F4906343F08B
:104708008003A38113E02A4600F080FB064670B9B7
:104718005046216900F0E0FA0C23CAF80030A3895A
:104728004FF0FF3043F04003A381BDE8F0872661D6
:104738003E4426604E466561ED1BA560B14500D23A
:104748004E4632462068414600F0ABFAA368002086
:104758009B1BA36023681E442660BDE8F087000009
:104768002DE9F0439DB003938B8906461C060D4640
:1047780090460CD50B6953B9402100F0F1FA286036
:10478800286110B90C233360CCE040236B6100230F
:10479800099320238DF8293030238DF82A30434699
:1047A8001C4613F8012B1AB9B4EB08090FD002E024
:1047B800252AF5D1F8E73046294642464B46FFF709
:1047C80075FF013000F0A980099B4B4409932378B9
:1047D800002B00F0A28000234FF0FF3204930793D0
:1047E800059206938DF853301A9304F10108444654
:1047F800DFF8489121784846052200F039FA08F197
:104808000108049B30B1C9EB000001228240134328
:104818000493ECE7D80644BF20228DF853201907EB
:1048280044BF2B228DF8532022782A2A02D00799D8
:1048380023460EE0039A0134111D12680391002AE1
:10484800BBBF524243F0020307920792B8BF0493DA
:104858000AE01C4622780133303A092A03D80A2094
:1048680000FB0121F5E7079123782E2B1AD16378F5
:104878002A2B0AD1039B02341A1D1B680392002BB2
:10488800B8BF4FF0FF3305930CE0611C00220C46C3
:1048980023780131303B092B03D80A2000FB023270
:1048A800F5E70592DFF8988021784046032200F06A
:1048B800DFF938B1049AC8EB000040238340134362
:1048C8000493013421781A48062204F101088DF86E
:1048D800281000F0CDF988B1164B33B9039B073384
:1048E80023F007030833039313E003AB0093304628
:1048F80004A92A46104BAFF3008007E003AB0093EE
:10490800304604A92A460C4B00F092F8421C074690
:1049180003D0099B3B44099341E7AB895B0601D46B
:10492800099801E04FF0FF301DB0BDE8F08300BFEB
:10493800184F000800000000B54600080E4F000898
:10494800144F00082DE9F84391461F468A680B6901
:1049580006469342B8BF1346C9F8003091F8432081
:104968000C46DDF8208012B10133C9F80030236805
:10497800990642BFD9F800300233C9F800302568DB
:1049880015F006051CD094F843302268003318BF90
:10499800012392061FD5E118302081F843005A1CE4
:1049A80094F845102244023382F8431013E030464D
:1049B800394604F119020123C047013007D00135F7
:1049C800E368D9F800209B1A9D42F0DBDBE74FF043
:1049D800FF30BDE8F8833046394604F14302C0474A
:1049E8000130F4D02268D9F80050E36802F00602DA
:1049F800042A08BF5D1B2269A3680CBF25EAE57578
:104A080000259342C4BF9B1AED184FF00009A94531
:104A18000ADA3046394604F11A020123C047013048
:104A2800D5D009F10109F2E70020BDE8F8830000BC
:104A38002DE9FF410C461746227E98466E2A064607
:104A48000A9B01F1430100F0B08012D8632A23D0F9
:104A58000AD8002A00F0BD80582A40F0CC8084F89B
:104A68004520DFF804E257E0642A1ED0692A1CD0EA
:104A7800C1E0732A00F0B18009D86F2A2ED0702ABD
:104A880040F0B980226842F0200222603FE0752A97
:104A980024D0782A3BD0AEE01A6804F14205111DF3
:104AA8001960136884F84230A9E020681A6810F089
:104AB800800F02D0101D186008E010F0400F02F1BE
:104AC8000400186002D0B2F9003000E01368002B2F
:104AD8003EDA2D225B4284F8432039E020681A68C8
:104AE80010F0800F02D0101D186007E010F0400F82
:104AF80002F10400186001D0138800E01368227ED8
:104B0800DFF864E16F2A0CBF08220A221CE0782231
:104B1800DFF858E184F845202268186812F0800F01
:104B280000F104051D6003D1550601D5038800E096
:104B38000368D00744BF42F0200222601BB92268F4
:104B480022F0200222601022002084F8430002E0B4
:104B5800DFF814E10A226568002DA8BF2068A56067
:104B6800A4BF20F00400206003B965B10D46B3FB73
:104B7800F2F002FB10331EF8033005F8013D03463E
:104B88000028F4D100E00D46082A0BD12368DA0783
:104B980008D5236962689A42DEBF302305F8013CD4
:104BA80005F1FF35491B21612EE025681A6815F0CB
:104BB800800F606903D0151D1D60136808E015F0AB
:104BC800400F02F104051D60136801D0188000E051
:104BD8001860002323610D4616E01A68111D19603C
:104BE800156800212846626800F042F808B1401BA9
:104BF8006060636804E004F1420584F84220012300
:104C08002361002384F84330CDF8008030462146E4
:104C180003AA3B46FFF796FE013002D14FF0FF3062
:104C28001FE0304639462A462369C0470130F5D08F
:104C380023689B0705D4E068039B9842B8BF1846D1
:104C48000FE00025E368039A9B1A9D42F3DA304689
:104C5800394604F119020123C0470130DED001357D
:104C6800F0E704B0BDE8F0811F4F0008304F00089E
:104C780010B5C9B202449042034605D01C780130F1
:104C88008C42F8D1184610BD002010BD10B5431E47
:104C98000A44914204D011F8014B03F8014FF8E798
:104CA80010BD814210B501EB020301D3421E0BE097
:104CB8009842FBD28118D21AD34204D013F8014D7E
:104CC80001F8014DF8E710BD994204D011F8014BE5
:104CD80002F8014FF8E710BD30B500293CD051F873
:104CE800042C0B1F1D49002AB8BF9B180A680C46E4
:104CF80012B95A600B6030BD93420DD2196858182A
:104D0800904201BF5A5852181A60426823605A608C
:104D180030BD994203D80A4651680029F9D1146870
:104D280015199D420AD11B682344D0188842136084
:104D380012D10868034413604B680CE002D90C23B5
:104D4800036030BD1C681819884201BF08684968AB
:104D5800001918605960536030BD00BFE0000020A2
:104D680070B5CC1C24F0030408340C2C38BF0C2478
:104D7800002C064603DA0C233360002070BD8C42F9
:104D8800F9D3204A136810461946A1B10A68121BC4
:104D98000ED40B2A03D90A608B188C501FE08B4263
:104DA8000BBF5A684A6802605A6018BF0B4616E083
:104DB8000B464968E9E7144D2B681BB9304600F0EB
:104DC8004BF828603046214600F046F8421C03465E
:104DD800D1D0C51C25F0030585420AD11C6003F11A
:104DE8000B001A1D20F00700821A0AD05142995070
:104DF80070BD3046E91A00F02FF80130BBD02B46C1
:104E0800ECE770BDE0000020DC000020F8B50746A4
:104E180015460E4621B91146BDE8F840FFF7A0BF78
:104E28001AB9FFF759FF2846F8BD00F025F8A8423F
:104E38000ED238462946FFF793FF044650B1314653
:104E48002A46FFF723FF38463146FFF745FF01E0C2
:104E58003046F8BD2046F8BD38B5064C0023054657
:104E68000846236000F012F8431C02D1236803B1FE
:104E78002B6038BDCC03002051F8040C0028BEBFBD
:104E8800091851F8043CC01804387047044A054909
:104E98001368002B08BF0B4618441060184670476B
:104EA800E4000020D0030020F8B500BFF8BC08BC1F
:104EB8009E467047F8B500BFF8BC08BC9E467047D0
:104EC80002030405060708090A0B0C0D0E0F101043
:104ED80001020000000000000000000001020304BD
:104EE800060708090000000001020304000002018F
:104EF8000405030025693B25693B25693B25690AAB
:104F08000D0000004300232D302B2000686C4C005E
:104F180065666745464700303132333435363738B1
:104F2800394142434445460030313233343536370F
:0C4F3800383961626364656600000000A7
:044F4400550200080A
:044F48002D0200082E
:104F4C0000A24A0464000000D0070000D007000053
:104F5C00D0070000D007000000002042D00700005E
:104F6C00D00700000000000000000000000000005E
:104F7C000000000000000000000000000000000025
:104F8C00000000000C4F00080000000000000000B2
:104F9C000000000000000000000000000000000005
:104FAC0000000000000000000000000000000000F5
:104FBC0000000000000000000000000000000000E5
:084FCC00000000002400002099
:04000005080045B5F5
:00000001FF
